:020000040800F2
:100000005821012085010008C901000811170008C6
:10001000C9010008C9010008C9010008000000006A
:10002000000000000000000000000000C9010008FE
:10003000C901000800000000C9010008C90100084A
:10004000C9010008C9010008C9010008C901000868
:10005000C9010008C9010008C9010008C901000858
:10006000C9010008C9010008C9010008C901000848
:10007000C9010008C9010008C9010008C901000838
:10008000C9010008C9010008C9010008C901000828
:10009000C9010008C9010008C9010008C901000818
:1000A000C9010008C9010008C9010008C901000808
:1000B000C9010008C9010008C9010008F9100008B9
:1000C00005110008111100081D110008C9010008E0
:1000D000C9010008C9010008C9010008C9010008D8
:1000E000C9010008C9010008C9010008C9010008C8
:1000F000C9010008C9010008C9010008C9010008B8
:10010000C9010008C9010008C9010008C9010008A7
:10011000C9010008C9010008C9010008C901000897
:10012000C9010008C9010008C9010008C901000887
:10013000C9010008C9010008C9010008C901000877
:10014000C9010008C9010008C9010008C901000867
:10015000C9010008C9010008C9010008C901000857
:100160002911000835110008C9010008C90100085B
:10017000C9010008C9010008C9010008C901000837
:04018000C9010008A9
:10018400002103E00A4B5B584350043109480A4BF1
:1001940042189A42F6D3094A02E0002342F8043B8B
:1001A400074B9A42F9D301F06FFE01F0FBFA704756
:1001B400E03700080000002030000020300000205C
:1001C40054010120FEE7000037B5012002F074FA63
:1001D400002401902546E0B200F046F801AA08B9CF
:1001E40010551DE0135D042B0BDD174800F07EF95C
:1001F400019800F082F90120002102F04DFA00205C
:1002040020E00133DBB2042B135509D90F4800F069
:1002140055F9204600F071F90D4800F067F9012501
:100224000134042CD7D1019C3CB10A4800F046F9B2
:10023400204600F062F900F0D1F80120214602F0D6
:100244002BFA284603B030BD74310008A0310008F1
:10025400AB310008B531000808B500F0A7FB80F009
:100264000100C0B208BD000008B5054B03EB001344
:100274005868198901F067FF003018BF012008BDD4
:10028400FC28000838B500242546E0B2FFF7ECFF4F
:10029400A04001340543042CEDB2F6D1284638BD04
:1002A40073B50020014602F04FF80120002102F04E
:1002B4004BF80220002102F047F84FF4804001215E
:1002C400104C02F085F904F14006684601F032FF53
:1002D40002238DF80530A37B60688DF80730002574
:1002E400A3688DF8045069461034009301F0EAFEC7
:1002F400B442EAD14FF48040294602F069F902B0D1
:1003040070BD00BFFC28000810B504460848402111
:1003140002F0D8FA0028F9D00548214602F0CEFAB6
:100324000348402102F0CEFA0028F9D010BD00BFE6
:10033400001001402DE9F043DFF89890DFF8988031
:1003440087B01020012102F043F948460921072211
:1003540001F004FF07210A4606AD404601F0FEFE07
:100364004FF4007345F8183D00240226012748463F
:1003740029468DF806408DF807708DF804608DF8D5
:10038400056001F09FFE80234046294600938DF8C6
:10039400046001F097FEADF80C40ADF80E40ADF8E6
:1003A4001040ADF8144004F1804404F58834084B3F
:1003B400029320460C2302A9ADF8123002F018FA79
:1003C4002046394602F06EFA07B0BDE8F08300BF5C
:1003D40040420F0000000240000402402DE9F043B7
:1003E400334D83B02C6804F12E0323F0070300AFD0
:1003F400ADEB030D50238DF8003021238DF801302F
:1004040000238DF8023003238DF8033004F1210317
:100414005BBAADF80430274B04F127086E460DF1A2
:10042400060203F11C0153F8040B42F8040B8B423F
:10043400F9D11B78137004F12309224606F1230035
:100444001D4902F045FA31464A46002001F0C4FC39
:1004540007F1080304F5927443F8040D186846F88C
:100464000900FE23B4FBF3F34344073323F00703EB
:10047400ADEB030D31464246684601F085FC044667
:100484005520FFF741FF6E466C44A64207D016F88C
:10049400010B552808BF0020FFF736FFF5E755206C
:1004A400FFF732FF00230C372B60BD46BDE8F08315
:1004B40030000020442900083400002010B5441EF8
:1004C40014F8012F7AB108490B68FF2B0BD80A2ABC
:1004D40002D1FFF783FFF3E70D2A1FBF581C5B18F7
:1004E40008601A71ECE710BD3000002008B5FFF772
:1004F400E5FFBDE80840FFF771BF1FB50C2201A955
:1005040001F09AFC01A8FFF7D9FF05B05DF804FBE0
:10051400014608B5044802F062F90348022102F0DA
:1005240060F90028F9D008BD003800402DE9F047F3
:1005340007310733089E099F92464FEAD108DD0828
:1005440081460024B4420CD004EB0A03122000FBC1
:100554000380494638442A4602F0BAF90134A944D2
:10056400F0E7BDE8F087000008B54FF480400121B2
:1005740002F022F805484FF40071012201F0E9FD70
:100584000720BDE8084001F047BC00BF000402405A
:1005940008B5072001F040FC4FF400710648002222
:1005A40001F0D7FD042001F037FC4FF48040002116
:1005B400BDE8084002F000B800040240F8B5074660
:1005C400FFF7D2FF8020FFF7A3FF0024661C30BA98
:1005D40090FAA0F0C0B2FFF79BFF122303FB047450
:1005E4000025605D00BA90FAA0F00135C0B2FFF7B3
:1005F4008FFF122DF5D10020FFF78AFFA82E344675
:10060400E4D10020FFF784FFBDE8F840FFF7C0BF46
:1006140010B5ADF6D83D02AC204600214FF43D6242
:1006240002F061F91B238DE8180010214022692390
:100634000448FFF77BFF2046FFF7C0FF0DF6D83DC7
:1006440010BD00BF612900082DE9F043ADF6DC3D83
:1006540002AC00214FF43D620546204602F043F906
:100664002C238DE818002B48182120225C231C27FA
:10067400FFF75CFFBE460F23BB402B4023FA07F273
:10068400254B242101FB0233002202EBC20000F6B9
:10069400280013F802C020440021082907D00126AD
:1006A4008E4016EA0C0F14BF0126002603E09E18A4
:1006B400767806F0010686B101EB0E06F6B24FEA33
:1006C400D6094FF0010806F0070608FA06F610F8F6
:1006D400098046EA080600F8096001310929DCD1DD
:1006E4000232242AD1D10EF10B0EBEF1740FA7F100
:1006F4000407C0D10E238DE81800102190226D2329
:100704000648FFF713FF2046FFF758FF0DF6DC3DC0
:10071400BDE8F083DB2A0008EB2C00082B2F00082F
:1007240008B5FFF721FF0020FFF7F2FE0020FFF7D6
:10073400EFFE0020FFF7ECFEBDE80840FFF728BFFE
:10074400F0B5214B1A685E246043B0FBF1F4944287
:10075400ADF6DC3D34D002AD00214FF43D622846B5
:100764001C6002F0C0F81B238DE8280017481021F4
:1007740040226923FFF7DAFE08238DE82800144895
:1007840018216A226023FFF7D1FE002000F286714F
:1007940029440022A2420DD002F11903DBB2DF0882
:1007A400012603F0070306FA03F3CE5D3343CB556A
:1007B4000132EFE712306C28E8D12846FFF7FEFE3D
:1007C4000DF6DC3DF0BD00BF0000002061290008EB
:1007D400EF2F00082DE9F843224E234CDFF88C90CC
:1007E4004FF48040012101F0E7FE30460A21052242
:1007F40001F0B4FC04F10408052230460F2101F095
:10080400ADFC3046414601F05DFC01254FF4007318
:100814000027304641466360A6F5E6362572A77286
:1008240001F050FC414648462572A772656001F00C
:1008340049FC304601F050FF304604F10C0101F050
:10084400A3FF3046294601F0BEFF484629462A4602
:1008540001F07FFC39464FF48040BDE8F84301F0D5
:10086400ABBE00BF000402400000002000000240B4
:10087400F0B50746ADF2044D0E460C460025B919F5
:10088400B4F5806FA1EB040168460DD94FF4806282
:1008940000F0C4F8284669464FF4806201F09CFADF
:1008A400A4F580640546EAE7224600F0B7F8284636
:1008B4006946224601F090FA0DF2044DF0BD08B5E8
:1008C400202001F0DFFD0028FAD108BD08B5022080
:1008D40001F0D8FD0028FAD00220BDE8084001F05C
:1008E400DBBD00B58DB0684601F055FD00230093D3
:1008F4004FF4807368460A9335230B9301F07CFD13
:10090400FFF7E4FFFFF7DBFF0DB05DF804FB000029
:1009140030B5022095B0012101F042FE00242248A6
:100924000021204403220B460C3400F0C3F8482C69
:10093400F5D101A801F026FD10230024019301A89C
:10094400162305930294039404940694079401F0E7
:1009540031FD012001F074FDFFF7C3FF08A801F089
:100964001AFD4FF44075662308A813930894129552
:1009740001F042FDFFF7AAFF08A801F00CFD99233E
:1009840008A813930894129501F036FDFFF79EFF13
:1009940042F6E06001F040FAFFF7A3FF022021468F
:1009A40001F0FEFD15B030BD5030000830B5012116
:1009B4008DB0022001F0F4FD022001F055FD6846DF
:1009C40001F0E9FC4FF0806300934FF0407304930F
:1009D4004FF4407368460A93AF230B9301F00CFD68
:1009E400FFF774FF01F048FD054601F045FD04469C
:1009F40001F042FD240244EA004040EA0504FFF706
:100A04005EFF0220002101F0CBFD0348231A584267
:100A140058410DB030BD00BFC225370070B5154632
:100A24008CB004460E460220012101F0B9FD681E77
:100A340001F01AFD684601F0AEFC4FF080630093AC
:100A44004FF040730493042305934FF440630993D8
:100A54004FF440730A934FF40053089368460B23F2
:100A64000B9301F0C9FC304601F0F6FC2544AC427E
:100A740004D001F001FD04F8010BF8E7022001F0B5
:100A84000BFDFFF71CFF0220002101F089FD0CB0D3
:100A940070BD0000024A136B43F0FF0313637047F9
:100AA40000380240024A136B23F0FF0313637047BC
:100AB4000038024013B504464068009002208DF8C7
:100AC40004008DF805208DF8061020682189A27A8B
:100AD4008DF8073001F042FB2068694601F0F2FA14
:100AE40002B010BD02460068838823F4E0631B044F
:100AF4001B0C838003889BB243F400730380082398
:100B04000020517513751076704707B500230091C6
:100B140069468DF804308DF805308DF8073001F002
:100B2400D1FA03B05DF804FB10B50B4C342300FB81
:100B34000344236B7BB10A2001F073F96068A16858
:100B4400FFF7E3FF20696169FFF7DFFF236B0120F3
:100B5400BDE81040184710BD98300008027D082AEF
:100B640010B5044607D10268938823F4C0631B04BC
:100B74001B0C938084E0434B006803EB8203596BA6
:100B840001F0BCFB00287BD0237D072B72D8DFE863
:100B940003F0040B1921323B5A6E237A226803F0C6
:100BA400FE03138201232DE02268A37A1382637A61
:100BB4000BB1022326E093889BB243F480639380B5
:100BC40006231FE0226813889BB243F480731380CA
:100BD400032317E0237A226843F001031382E37AA4
:100BE400012B01BF138823F480631B041B0C08BF73
:100BF4001380042306E0226893889BB243F4806345
:100C04009380052323753BE023682269198A237B9B
:100C1400D154237BE27A0133DBB2591C9142237312
:100C240007D12268138823F480631B041B0C1380F0
:100C340026E0934224D12268938823F480631B0422
:100C44001B0C938013E0237B21692268CB5C138205
:100C5400237BE17A0133DBB29942237310D1938869
:100C640023F480631B041B0C93800723CAE72046EC
:100C7400012101E020460021BDE81040FFF732BF0A
:100C8400002010BD983000082DE9F341184C34239E
:100C940000FB0344236B43B300209847D4F804803B
:100CA400A668009600250127404669468DF8047021
:100CB4008DF805508DF8075001F004FAB1B22A46B8
:100CC400404601F046FA2669646900943046694654
:100CD4008DF804708DF805508DF8075001F0F2F985
:100CE4003046A1B22A4601F034FA02B0BDE8F081E0
:100CF400983000081C23104A434370B505460F4C36
:100D0400D058D61801F03CFA342305FB03440021E3
:100D1400E06901F051FC337923B92846BDE87040FD
:100D2400FFF7B2BF6068A168FFF7EFFE2069616951
:100D3400BDE87040FFF7E9BE340100209830000898
:100D44002DE9F04F344D1C2303FB005387B01B796E
:100D540007460BB9FFF7E8FE304B342407FB043495
:100D64000226D4F80490A389A26894F80EB00193E3
:100D74004FF001084FF0000A484602A902928DF88C
:100D84000C608DF80D608DF80E808DF80FA001F0C9
:100D940099F9019B484619465A4601F0DFF9D4F8FF
:100DA4001090238B626994F81AB00193484602A903
:100DB40002928DF80C608DF80D608DF80E808DF820
:100DC4000FA001F07FF9019B5A461946484601F0ED
:100DD400C5F94146E06901F0EFFB02A801F068FAA9
:100DE4000F4A236A029393424FF48063ADF81230A2
:100DF4004FF01C0384BF626AADF80E2003FB07F4B6
:100E040002A9285901F0EAF92859012101F05EFAF2
:100E140007B0BDE8F08F00BF34010020983000080F
:100E2400A08601002DE9F341414C9846237F0546F5
:100E34000E4617461BB93F484FF4BD7103E020B17D
:100E44003C4840F27B1100F079FF23790BB9002074
:100E54006AE023681B8B9B0711D49DF82030E37252
:100E64000025099B277284F80A806672257325750C
:100E74002361E5822068012101F034FA1FE0FFF7C5
:100E840039FF2846FFF75CFF22682B48138B99072C
:100E9400E3D50138FAD1DAE7227E22B1019A511E54
:100EA4000191002AF8D100222276019A204902B346
:100EB4000A7D082A13D14D7D237D082B26D0236873
:100EC4001A8892B242F480721A809A8892B242F4DA
:100ED40040729A8001222276174A0192DEE7CA8A7A
:100EE400B2F57A7F05D20132CA82012000F099FF5F
:100EF400E2E79A8822F4E0621204120C9A801A88BB
:100F040092B242F400721A8008230B7522680A4CCC
:100F1400138B9B0707D5013CFAD12046FFF7EAFE65
:100F24002046FFF70DFF284602B0BDE8F08100BF60
:100F340034010020F531000880841E00017D03681F
:100F4400082906D19A8822F480721204120C9A801D
:100F540038E09A8A120541BF9A8A22F40062120488
:100F6400120C48BF9A829A8AD20541BF9A8A22F407
:100F740080721204120C48BF9A829A8A52051ED5B6
:100F84009A8A22F480621204120C04299A820AD1E9
:100F9400032202759A8822F4E0621204120C9A80E9
:100FA400002303760EE0012909D19A8822F4E06235
:100FB40012040021120C01759A80017602E00021CE
:100FC400FFF790BD0020704737B5124C124B2360D9
:100FD40008222275482200238DF8042001250C22C2
:100FE40001A88DF80520237123762373E37223610E
:100FF4008DF806308DF8075000F082FF492301A8D0
:101004008DF8043000F07CFF206801F0B9F82577F2
:1010140003B030BD34010020005C004013B50D4C1A
:10102400227F034622B90C484FF48C7100F086FEEF
:1010340038B1012200920848084A4FF48D7100F03B
:1010440071FE23790BB9FFF77BFE237901332371FA
:1010540002B010BD34010020F53100080A32000846
:101064000C4A117F08B519B90B484FF4957103E088
:1010740020B1094840F22B1100F060FE13793BB116
:10108400013BDBB213711BB9BDE80840FFF732BE68
:1010940008BD00BF34010020F531000837B50D4606
:1010A40014460093069B019301212A462346FFF729
:1010B400B9FE03B030BD07B500930123FFF7EEFF7F
:1010C40003B05DF804FB37B50D4614460093069B48
:1010D400019300212A462346FFF7A4FE03B030BD46
:1010E4001FB504AC04F8013D01230094FFF7EBFFA6
:1010F40004B010BD0148FFF731BD00BF340100202A
:101104000148FFF71BBF00BF340100200148FFF76F
:1011140025BD00BF500100200148FFF70FBF00BFED
:10112400500100200148FFF719BD00BF3401002021
:101134000148FFF703BF00BF3401002038B50C4657
:1011440005460020FFF76AFF234681212A46002036
:10115400FFF7B1FF04460020FFF782FF204638BDA9
:1011640038B50C4605460020FFF758FF234680217A
:101174002A460020FFF7B4FF04460020FFF770FF63
:10118400204638BD37B50D460DF107010446FFF77B
:10119400D5FF50B19DF807300121A9401943C9B2C8
:1011A40020468DF80710FFF7DBFF03B030BD0000C9
:1011B40013B590200DF10701FFF7C0FF044648B3B3
:1011C4009DF80740A4F111035C425C4114B3FF2174
:1011D4004220FFF7C5FFFF214120FFF7C1FF352063
:1011E4000DF10701FFF7AAFF044620B90B480C4A8A
:1011F400BE2100F097FD9DF80710352041F0030152
:101204008DF80710FFF7ACFF0A201E21FFF7A8FF97
:101214000028EBD0204602B010BD00BF36320008D3
:101224005432000807B587200DF10701FFF786FF48
:1012340018B19DF80700C0F3800003B05DF804FB0B
:1012440007B536200DF10701FFF778FF20B19DF8AF
:1012540007301B090B2B01D0002014E077200DF17F
:101264000701FFF76BFF0028F6D09DF8073003F065
:10127400100303F0FF0023B1FFF7D4FF80F0010057
:10128400C0B200F0010003B05DF804FB08B53620DD
:101294000121FFF777FF00B1FEE708BD07B5EF2195
:1012A4007420FFF75DFFFF217520FFF759FF0DF153
:1012B40007017720FFF742FF0DF107017820FFF7C0
:1012C4003DFF0A213920FFF74BFF35200421FFF7AA
:1012D40059FF00B1FEE703B05DF804FBB0F1006F05
:1012E40010B504460BD20C48FFF7E8F82046FFF788
:1012F40004F90A48FFF7FAF84FF0FF3010BD084B25
:10130400002053F8042BA24202D81A68944202D354
:1013140001300B28F5D110BDB43200087332000837
:10132400EC3000082DE9F8430446174699460E466A
:10133400C1B3FFF7D3FF0546601E3044FFF7CEFF6D
:10134400002D804631DB00282FDB461B01361FB100
:10135400002031464A46B84700F014FE2C46444566
:101364001EDCF32000F024FE114B002133F814009E
:1013740000F056FE09280AD00E48FFF79FF82046D1
:10138400FFF7BBF8FFF72AF800F00AFE0DE02FB1D3
:10139400C5F10100204431464A46B8470134DEE72E
:1013A40000F0FEFD0120BDE8F8830020BDE8F883CD
:1013B4001C3100088C3200082DE9F0470E46154612
:1013C4000746984600F0DEFDF32000F0F1FD4FEAF9
:1013D400D51934463544AC42C6EB040A20D0B81BB8
:1013E400204414F8011B00F051FE09280CD00F48CA
:1013F400FFF764F83846FFF780F8FEF7EFFF00F0D8
:10140400CFFD0020BDE8F087B8F1000FE3D01AF05B
:101414007F0FE0D14FEADA104946089AC047DAE76D
:1014240000F0BEFD0120BDE8F08700BFA432000833
:1014340008B545F2555000F06FFF042000F072FF2C
:1014440040F6FF7000F074FF002000F065FF4FF4D9
:1014540080500121BDE8084000F088BD08B57D201A
:1014640001F0FEF8003018BF012008BD4900FFF765
:1014740067B900002DE9F041012186B0054600203E
:10148400FFF75EF9042000F0A1FB03A8294600F051
:10149400FBFB03A800F007FC08B93C4814E03C48F7
:1014A4000C35FFF723F804992846FFF7E1F90446C1
:1014B4003848FFF703F82046FFF71FF8FEF78EFFC2
:1014C400059B9C4204D03448FFF710F8012059E0F2
:1014D400049C3248FFF70AF82146314A3148002378
:1014E400FFF720FF3048049FFFF700F84FEA570842
:1014F4000024BC4220D23E1BB6F5803F28BF4FF4E7
:1015040080362A4861193246FFF788FA002304F12D
:101514000060009300F5804024493246FFF74CFFF9
:1015240018B92348FEF7E2FF06E0344408EB540000
:101534003946FFF705F9DCE71E48FEF7BFFF0498BC
:10154400FEF7DBFF1C48FEF7B9FF1649049A00209A
:1015540000F042FC04461948FEF7B0FF0598FEF778
:10156400CCFF1748FEF7AAFF2046FEF7C6FFFEF79A
:1015740035FF059B9C4204D01248FEF7B7FF0220BA
:1015840000E0002006B0BDE8F08100BFBD320008D5
:10159400DB320008F83200080E330008313300084B
:1015A4007114000800400008443300085101002071
:1015B4005733000862330008703300087933000899
:1015C4008C3300089233000810B5022000F016FB9B
:1015D400D8B3042000F012FB044670B11B48FEF798
:1015E40085FF042000F0FEFA022000F0FBFA4FF41D
:1015F4000040BDE8104000F0F5BA1548FEF776FF4C
:10160400082000F0EFFA102000F0ECFA202000F09F
:10161400E9FA402000F0E6FA2046FFF72BFF022803
:1016240007D1082000F0D2FA102000F0CFFA00F021
:10163400A1FB042000F0D6FA022000F0D3FA4FF404
:101644000040BDE8104000F0C1BA10BDDD33000811
:101654001334000810B52548FEF748FF4FF4001076
:10166400FFF708FF10B102283AD809E0202000F063
:10167400B9FA402000F0B6FA802000F0A7FA2FE073
:10168400082000F0A3FA102000F0A0FA202000F0B7
:10169400B5FA20B91648FEF729FF202007E04020BC
:1016A40000F0ACFA58B91348FEF720FF402000F0D0
:1016B4008DFA4FF4007000F089FA00F05BFB0E48DD
:1016C400FEF714FF082000F08DFA102000F08AFACB
:1016D400202000F087FA402000F084FA002400E083
:1016E4000124042000F07EFA204610BD2E340008A8
:1016F4004834000881340008BA34000808B50248A8
:10170400FEF7F4FE00F0BEFAF43400081EF0040FF5
:101714000CBFEFF30880EFF30980FFF7EFBF7047CA
:1017240008B50120FEF7A0FD08B900200FE0002055
:10173400FEF79AFD0028F8D00220FEF795FD002858
:10174400F3D00320FEF790FD80F00100C0B200F05A
:10175400010008BD1FB504461048FEF7C7FE01A9E5
:101764000C22204600F068FB01A8FEF7BFFE2046CD
:10177400FEF76AFFFEF786FD094B20F0040018709F
:101784001C46FEF77FFD237800F0FB00834201D066
:1017940000F0F0FA0A2000F044FBF2E7EA34000813
:1017A4005101012030B585B0FFF774F94FF0805036
:1017B400012100F001FF022000F0D2FD012807D131
:1017C400022000F0D7FDA548FEF790FE00F0D9FAFC
:1017D40000214FF0805000F0EFFEFEF7ABFDA04873
:1017E400FEF784FE9F48FEF781FE9F48FEF77EFECB
:1017F4009E48FEF77BFE9E48FEF778FE9848FEF76B
:1018040075FEFFF7E1FB9B48FEF770FEFFF7D0FC87
:101814009948FEF76BFE00F0FBF99848FEF766FE68
:1018240000F022FA00210C2201A801F05CF800F07B
:1018340017FA01A90C2200F0FFFA01A8FEF756FEE0
:101844008748FEF753FE8648FEF750FE4FF480406B
:1018540000F0D4F990B18A48FEF748FE4FF4804076
:1018640000F0C0F9082000F0BDF9102000F0BAF92A
:10187400202000F0B7F9402000F0B4F9FFF7E0FCB5
:1018840038B18048FEF732FE7F48FEF72FFEFFF79F
:1018940005FDFFF73DF8FEF703FDFEF79BFFFEF79E
:1018A400B7FEFEF791FC08B1784803E0FEF7D4FCDC
:1018B40010B17748FFF74EFF00F0C2F9802000F026
:1018C4009DF918B1802000F08DF949E04FF4003003
:1018D40000F094F920B14FF4003000F083F959E19D
:1018E400FFF71EFF68B16B48FEF700FE41F2883433
:1018F400FFF716FF78B1012000F093FA013CF7D10D
:1019040048E1654B0CCB013301D0013203D163486C
:10191400FEF7ECFD3EE1FFF7A1FD18B3FFF79EFDD6
:1019240010B15F48FEF7E2FD4FF4007000F066F975
:1019340010B15C48FEF7DAFD4FF4007000F052F984
:10194400102000F05BF9D0B15748FEF7CFFD082016
:1019540000F048F9102000F045F9FFF77BFEF8B9D4
:101964005248A7E74FF4007000F048F90028D5D199
:10197400082000F037F9102000F034F90EE00820B8
:1019840000F03CF920B14A48FEF7B0FD102003E016
:101994004848FEF7ABFD082000F018F9FFF714FEE5
:1019A4004FF4005000F02AF904464FF4805000F040
:1019B40025F9400040EA8400C4B24FF4006000F00E
:1019C4001DF92043C0B20728C3B20DD14FF4006003
:1019D40000F008F94FF4805000F004F94FF400507F
:1019E40000F000F9344865E70133DBB2023B4FF401
:1019F4000060052B11D8DFE803F00C1003100C1065
:101A040000F0F0F84FF4805000F0ECF84FF4005080
:101A140003E000F0E7F84FF4805000F0D7F84FF4FB
:101A2400002000F0EBF8002851D04FF4002000F023
:101A3400D9F82248FEF75AFD0024FFF7F3FB0028EB
:101A440040D0042C03D11E48FEF750FD00244FF46F
:101A5400FA7000F0E6F90134EFE700BFFF34000844
:101A6400403700080C3500081D3500082E350008E5
:101A74003F350008503500085B350008673500081D
:101A8400703500089D350008CE350008014550FE2C
:101A9400024550FEED3500080040000828360008D5
:101AA4003B3600085336000873360008034550FEE1
:101AB4009B360008C1360008044550FEE73600088E
:101AC400FB3600083548FEF711FDFFF7DFFBFFF793
:101AD400AFFCFEF7E7FF324B32485C681D68FEF747
:101AE400EDFC2046FEF709FD2F48FEF7E7FC002237
:101AF400930003F1604303F5614301324FF0FF317A
:101B0400082AC3F88010C3F88011F1D1274B284A62
:101B1400196B0A401A635A6B22F0C0025A639A6B1B
:101B240022F003029A63196C224A0A401A64596C1F
:101B3400214A0A405A6400F0B5FC2048012100F013
:101B440053FD1E48002100F04FFDF120012100F05B
:101B540057FDF120002100F053FD0120014600F063
:101B64005BFD0120002100F057FD1548012100F024
:101B74005FFD1348002100F05BFD1248012100F0D5
:101B840063FD1048002100F05FFD63B64FF0FF3E97
:101B9400AD4620470C48FEF7A9FCDEE616370008E0
:101BA4000040000825370008393700080038024093
:101BB40000EF9FFF003619E8CC86E8FE0010E02213
:101BC400FFC9FEF6337F77044137000810B5044699
:101BD400002000F071FD40EA04010020BDE810403F
:101BE40000F05ABD10B50446002000F065FD20EA5F
:101BF40004010020BDE8104000F04EBD10B50446BD
:101C0400002000F059FD204214BF0120002010BD27
:101C140008B501214FF0805000F0CEFC012000F007
:101C24008DFB4FF08050002100F0C6FC0120FFF72F
:101C3400E5FF20B90121BDE8084000F02DBD08BD35
:101C440008B50648FEF73AFC002000F035FDFEF723
:101C540054FCBDE80840FEF7C1BB00BF6037000874
:101C6400022000F029BD000008B5FFF7F9FF044980
:101C7400884204D00220BDE8084000F00DBD08BD34
:101C84008BB8185800BEFDE71FB504460C2201A806
:101C9400FEF7C4FE01AB03CB20601868A0602046A9
:101CA400616004B010BD0068A0F10C0358425841B3
:101CB4007047000080B50646174610480D461C467E
:101CC400FEF7FCFB3846FEF7F9FB0D48FEF7F6FB82
:101CD4003046FEF7F3FB0B48FEF7F0FB2846FEF711
:101CE4000CFC2CB10848FEF7E9FB2046FEF7E6FBA6
:101CF4000648FEF7FBFBFFF7C5FF00BF6C37000883
:101D04001A350008753700081B35000840370008ED
:101D14001FB506AA52F8044B039200921A462346B2
:101D2400FFF7C8FF0CB41FB506AA52F8043B039290
:101D34000092014AFFF7BEFF7737000807B500237A
:101D440000937246014BFFF7E3FF00BF7E370008A4
:101D5400BFF34F8F0549064BCA6802F4E062134390
:101D6400CB60BFF34F8F00BFFDE700BF00ED00E085
:101D74000400FA0508B5FEF7D3FC00F085FCFFF774
:101D8400E7FF08B5FFF7E4FFF0B50646002401209D
:101D94002546034694421DD011F804C000F1010EFB
:101DA400BCF1000F03D17355774605460DE00133AE
:101DB400DBB2FF2B774606F800C007D102F1FF3CE7
:101DC400644506D07355871C754601230134384693
:101DD400E0E770467355F0BD30B5C9B1C0430A445D
:101DE400914213D011F8013B0A4D83EA000404F038
:101DF4000F0455F8244084EA101080EA131303F00A
:101E04000F0355F8233083EA1010E9E7C04330BDCF
:101E1400084630BD34310008062358430138FDD14B
:101E2400704710B504462CB14FF47A70FFF7F4FFF5
:101E3400013CF8E710BD00000A2A10B504DC114883
:101E4400BDE81040FEF752BB0C46302304F8023BB9
:101E540078234B701C220F2393400340D340092B5B
:101E640001D8303302E00F2B02D85733DBB200E045
:101E74002023043A04F8013B131DECD100238B7298
:101E840010BD00BFCA3700081949D1F8883043F49F
:101E94007003C1F88830174B1A68002042F0010221
:101EA4001A6098601A6822F0847222F480321A60F0
:101EB400114A5A601A6822F480221A60D8601A6C97
:101EC4000E4842F080521A64026842F440420260B2
:101ED4009A689A609A689A609A6842F480529A6002
:101EE4004FF4C062C3F800244FF000638B60704766
:101EF40000ED00E000380240103000240070004083
:101F0400C278037810B512B3164AD1684278C9432F
:101F1400C1F30221C1F10404E4B2A240D4B20F22FD
:101F24000A4181780A40224303F1604303F5614387
:101F34001201D2B283F8002303780122590903F075
:101F44001F0302FA03F3084A42F8213010BD5A096C
:101F5400012103F01F03994002F12003024A42F8D1
:101F6400231010BD00ED00E000E100E0044B9A688E
:101F740009B1104301E022EA00009860704700BFF5
:101F8400002004E0044B1A69002ABFBF034A5A60C8
:101F940002F188325A607047003C024023016745D1
:101FA400024A136943F0004313617047003C024046
:101FB400014BD860704700BF003C02400E4BDA680A
:101FC400D20310D4DA68D1060FD4DA68D2050ED45D
:101FD400DA6812F0E00F0CD1DB6813F0020F14BFC3
:101FE400082009207047012070470620704702200E
:101FF40070470720704700BF003C024007B5092323
:102004008DF80730FFF7DAFF8DF807009DF80730E9
:10201400012BF7D09DF8070003B05DF804FB000026
:1020240070B5064641B1012908D002290CBF4FF40E
:1020340000754FF4407503E00D4601E04FF48075E0
:10204400FFF7DCFF09281ED10F4C236923F44073EA
:102054002361216929432161236923F0F803236162
:10206400236943F002031E432661236943F480334A
:102074002361FFF7C3FF236923F00203236123696C
:1020840023F0F803236170BD003C024070B505469F
:102094000E46FFF7B3FF092811D1094C236923F435
:1020A4004073236123692361236943F0010323619E
:1020B4002E70FFF7A3FF236923F00103236170BD92
:1020C400003C0240F0B50E6800220123934003EA6D
:1020D400060E9E452AD1550003230468AB40DB431A
:1020E4001C4004600C79076804FA05FC013C4CEAC6
:1020F4000707012C076011D884684F791C4084605D
:102104008468AF4027438760446824EA0E0444602F
:102114008C7947689440A4B23C434460C46823402B
:10212400C360CB79C468AB402343C3600132102A37
:10213400CBD1F0BD4FF6FF730360002303714371ED
:102144008371C37170470369194214BF01200020D1
:1021540070470AB1018370474183704701F0070358
:10216400C90800EB810010B59B00046A0F21994057
:1021740024EA01010162016A9A401143016210BD1F
:1021840008B5134B984207D14FF40010012100F019
:102194004FFA4FF4001014E00E4B984207D14FF45D
:1021A4008000012100F044FA4FF4800009E00A4B5A
:1021B40098420BD14FF40000012100F039FA4FF49A
:1021C40000000021BDE8084000F032BA08BD00BF9D
:1021D4000054004000580040005C00407FB58688F1
:1021E40026F03F060446360468460D46360C00F0D9
:1021F40075F9029A2C48B2FBF0F081B20E43A68026
:1022040023882A4E23F001031B041B0C23802B6814
:10221400B3420AD85B000131B2FBF3F39BB2032B48
:1022240089B298BF0423218423E0EE884BF6FF7122
:102234008E421BBF19214B4303EB4303B2FBF3F361
:1022440015BF9BB2B2FBF3F343F480439BB2C3F3D9
:102254000B020AB943F001034FF4967101FB00F23B
:102264004FF47A7192FBF1F2013292B243F40043DB
:102274002284A38323886989AA889BB243F001033B
:102284002380238823F4816323F002031B040A437D
:102294001B0C13439BB223802A89AB8913439BB243
:1022A400238104B070BD00BF40420F00A08601002E
:1022B40041F288330360002383804BF6FF7203816D
:1022C40043814FF48043C28083817047038819B1EE
:1022D4009BB243F0010303E023F001031B041B0C36
:1022E40003807047038819B19BB243F4806303E011
:1022F40023F480631B041B0C03807047838A9AB207
:10230400038B10B542EA034321F07F4404EA03003F
:10231400431A5842584110BD014B1860704700BF22
:1023240000300040014B5860704700BF003000404F
:10233400014B9860704700BF00300040014B1860AB
:10234400704700BF20000E4210B9034B196070475C
:10235400024B1960704700BFA0000E429C000E4261
:10236400034B5B68184214BF01200020704700BF74
:1023740000700040024A136843EA8000106070470E
:10238400007000400023036043608360C360036106
:10239400436183617047002343608360C3600360CB
:1023A400036143618361C361036243628362C36205
:1023B400704700000E4903680A6810B544691C435D
:1023C40083691C4322F07F4323F030034268234394
:1023D40043EA02630B60C36882684C681A43054B86
:1023E40023401343026943EA02434B6010BD00BF1C
:1023F400001000A0FEF7E0FF90E80C001A43836889
:102404000D491A43C3681A4303691A4383691A437B
:10241400C3691A43036A1A43436A1A43836A1A4311
:10242400C36A10B51A434C69044B234013434269F1
:1024340043EA82434B6110BD001000A0000080906D
:10244400044B1A6810B142F0010201E022F00102CB
:102454001A607047001000A0024B9A68920658BF99
:1024640098617047001000A0024B9A68920658BF0A
:1024740018617047001000A0014B1878704700BF26
:10248400201000A0034B9B68184214BF01200020B9
:10249400704700BF001000A0014BD860704700BF18
:1024A400001000A00B4B1A68002142F001021A60D0
:1024B40099601A6822F0A85222F410221A60064A7F
:1024C4005A601A6822F480221A60D960C3F88C100A
:1024D400704700BF00380240103000242C4B9A682B
:1024E40002F00C0210B50C2A38D8DFE802F03737B6
:1024F400373707373737093737371E00254B2EE074
:102504005968234A5B6811F4800F03F03F03516854
:1025140014BF204A204AB2FBF3F31D4A5268C1F3A8
:1025240088114B43C2F3014213E05968184A5B68AF
:1025340011F4800F03F03F03516814BF154A164A83
:10254400B2FBF3F3124A5268C1F388114B43C2F34E
:10255400027201325200B3FBF2F300E00E4B0C4A5C
:10256400036093680D49C3F30313CC5C0368E34031
:1025740043609468C4F382240C5D23FA04F48460F9
:102584009268C2F342328A5CD340C36010BD00BF7C
:102594000038024000127A000024F4001E000020DB
:1025A400044B9A6B09B1104301E022EA00009863DE
:1025B400704700BF00380240044B1A6C09B1104345
:1025C40001E022EA00001864704700BF00380240AE
:1025D400044B5A6C09B1104301E022EA000058642C
:1025E400704700BF00380240044B1A6909B1104318
:1025F40001E022EA00001861704700BF0038024081
:10260400044B5A6909B1104301E022EA0000586101
:10261400704700BF00380240044B9A6909B1104367
:1026240001E022EA00009861704700BF00380240D0
:10263400044B1A6A09B1104301E022EA000018624F
:10264400704700BF00380240044B5A6A09B1104376
:1026540001E022EA00005862704700BF00380240DF
:102664004209012A074B01D11B6803E0022A0CBF6F
:102674001B6F5B6F00F01F0023FA00F000F00100F5
:10268400704700BF00380240024A536F43F0807322
:10269400536770470038024082B000230193054B12
:1026A4000193019B03EB80000190019B196002B030
:1026B400704700BF5028004082B000230193054BAF
:1026C4000193019B03EB80000190019B186802B009
:1026D400704700BF5028004008B5254B984207D1E9
:1026E4004FF480500121FFF7AFFF4FF4805039E0E1
:1026F400204B984207D14FF480400121FFF798FF07
:102704004FF4804009E01C4B98420BD14FF4004039
:102714000121FFF78DFF4FF400400021BDE8084080
:10272400FFF786BF154B984207D14FF400500121A3
:10273400FFF78AFF4FF4005014E0114B984207D181
:102744004FF480100121FFF77FFF4FF4801009E060
:102754000C4B98420BD14FF400100121FFF774FF8A
:102764004FF400100021BDE80840FFF76DBF08BD1D
:102774000030014000380040003C0040003401407B
:10278400005001400054014003884A8810B503F406
:1027940041540B8813438A881343CA8813430A8914
:1027A40013434A8913438A891343CA89134323432E
:1027B4009BB20380838B23F400631B041B0C838371
:1027C4000B8A038210BD038819B19BB243F0400306
:1027D40003E023F040031B041B0C0380704781813A
:1027E40070470389194214BF01200020704700007C
:1027F4007FB5038ACA889BB223F4405313430382F0
:1028040083890E469BB223F4B053098923F00C024A
:10281400B3880B4371890B439BB213438381838A2F
:10282400B2899BB223F440731343838204466846FF
:10283400FFF754FE1A4B9C4203D003F580639C427D
:1028440001D1039D00E0029DA38931681BB2002BD6
:102854004FF0190202FB05F2B4BF4D008D00B2FB2C
:10286400F5F5A2896426B5FBF6F00001010912B260
:10287400002A06FB1153ADBF1A01D900323132329E
:10288400B5BFB1FBF6F2B2FBF6F302F0070203F0B8
:102894000F03B4BF1043184380B2208104B070BD4D
:1028A40000100140838919B19BB243F4005303E043
:1028B40023F400531B041B0C83817047C1F30801EC
:1028C400818070470388194214BF0120002070479B
:1028D40010B5431E0A44914204D011F8014B03F889
:1028E400014FF8E710BD02440346934202D003F8B7
:1028F400011BFAE770470000E131000800080240BC
:1029040000200000020D0000E6310008000C024027
:102914000400000003020200E9310008001C024028
:102924000100000007000200F0310008001C024012
:102934000200000007010200000000000000000087
:1029440001424F4F544C4F41444552000000000097
:10295400002A2A000000000000000000000000001F
:1029640000006000000300180000000000000000E8
:102974006000000300180000000000000000600078
:1029840000030018000000000000000060000003C5
:1029940000180000000000000000600000030018A0
:1029A40000000000E003001F60F800C30718C00720
:1029B4000000F80FC07F60FE03F31F18F01F000033
:1029C4000C1860C06003061B301818300000063075
:1029D4003080E1010C0F60180C60000003601800E7
:1029E400E3001807C01806C0008001400C00620014
:1029F400100380180380008001C00C0066003003BF
:102A040080190380018001C0FCFF67003003801936
:102A1400FFFF018001C0FCFF630030038019FFFF4A
:102A2400008001C00C0060003003801903000080A6
:102A340001C00C00600030038019030000800140D5
:102A44000C006200100380180380008003601800EB
:102A5400C3001806C01806C000800730308081010A
:102A64000C0C60180C6000800D1860C00003061880
:102A7400303818300080F90FC07F00FE03F01F705B
:102A8400F01F0080E103001F00F800C00760C007CA
:102A94000080010000000000000000000000008031
:102AA40001000000000000000000000000800100A0
:102AB4000000000000000000000000800100000091
:102AC4000000000000000000008001000000000081
:102AD40000000000000000000C0006000000006080
:102AE4000030000018000300000000C000180000BF
:102AF4003080010000000080010C000060C0000074
:102B04000000000003060000C06000000000000098
:102B14000603000080310000000000008C0100006A
:102B2400001B000000000000D8000000000E0000A0
:102B34000000000070000000000E00000000000013
:102B440070000000001B000000000000D80000001E
:102B540080310000000000008C010000C060000013
:102B6400000000000603000060C000000000000038
:102B7400030600003080010000000080010C00000A
:102B840018000300000000C0001800000C0006003C
:102B940000000060003000000000000000000000A1
:102BA4000000000000000000000000000000000021
:102BB4000000000000000000000000000000000011
:102BC4000000000000000000000000000000000001
:102BD40000000000000000000000000000000000F1
:102BE40000000000000000000000000000000000E1
:102BF400000000000000000000000080FFFF010052
:102C040000000000000000FEFFFF7F000000000045
:102C14000000E07F0000FE07000000000000FE014D
:102C24000000807F0000000000801F00000000F80A
:102C34000100000000F00100000000800F0000000F
:102C4400007C0000000000003E000000000F0000B7
:102C540000000000F00000008003000000000000FD
:102C6400C0010000E00000000000000000070000B8
:102C74007000000000000000000E000018000000BA
:102C840000000000001800000C000000000000001C
:102C9400003000000600000000000000006000009A
:102CA400030000000000000000C0008001000000DC
:102CB40000000000008001C00000000000000000CF
:102CC4000000036000000000000000000000063067
:102CD400000000000000000000000C1000000000D4
:102CE400000000000000087C00FE00FF01C701C7CF
:102CF40001C701C701C701C701C701C701C701C790
:102D040001C701C701FF01FE007C0038003C003E02
:102D1400003E0038003800380038003800380038E9
:102D2400003800380038003800FE00FE00FE007C49
:102D340000FE00FF01C701C701C001C001E000F0AF
:102D44000078003C001E000E000F000700FF01FF8A
:102D540001FF017C00FE00FF01C701C701C001C0E3
:102D640001F8007800F800C001C001C001C701C724
:102D740001FF01FE007C00E000E000F000F000F83C
:102D840000F800F800FC00EC00EE00E600FF01FF94
:102D940001FF01E000E000E000E000FF00FF00FFB1
:102DA400000700070007007F00FF00FF01C701C004
:102DB40001C001C701C701C701FF01FE007C007CFF
:102DC40000FE00FF01C701C701070007007700FFED
:102DD40000FF01C701C701C701C701C701FF01FE09
:102DE400007C00FF01FF01FF01E000E000700070C3
:102DF40000700038003800380038001C001C001C2B
:102E0400001C001C001C007C00FE00FF01C701C761
:102E140001C701C701FE007C00FE00C701C701C74E
:102E240001C701C701FF01FE007C007C00FE00FF1A
:102E340001C701C701C701C701C701FF01FE01DCCA
:102E440001C001C001C701C701FF01FE007C0000F1
:102E5400000000000000007C00FE00FF01C701C765
:102E640001F001FC01CE01C701C701E701FF01DF49
:102E740001CE010700070007000700E700F701FF84
:102E840001CF01C701C701C701C701C701C701CFEE
:102E940001FF01F701E70000000000000000007CD2
:102EA40000FE00FF01C701C7010700070007000774
:102EB40000C701C701FF01FE007C00C001C001C0C2
:102EC40001C001CE01DF01FF01E701C701C701C74E
:102ED40001C701C701C701E701FF01DF01CE0100FE
:102EE400000000000000007C00FE00FF01C701C7D5
:102EF40001C701FF01FF010700C701C701FF01FE70
:102F0400007C00E000F000F8003800FE00FE00FE47
:102F140000380038003800380038003800380038ED
:102F2400003800380038000000068301000000006B
:102F340000000000000000068301000000000C00F7
:102F44000000000000068301000000000C000000E7
:102F540000D878369B79C0E3D90C8C67DB3C1BF82E
:102F6400FD7EBFFDE0F7FB1FC6EFFB7E1F98CD661D
:102F7400B3CD60369B19C66C18660398FD66B3FD25
:102F840060309B19C66F18660398FD66B3FD603008
:102F94009B19C36F186603980D66B30D60369B19B1
:102FA400C360186603F8FD7EBFFDECF79B19C36F81
:102FB400187E03D878369B79CCE399998167183CBD
:102FC4000318000000000000008001000000001849
:102FD40000000000000000000000000000180000D5
:102FE4000000000000000000000000FFFFFFFFFFE2
:102FF400FFFFFFFFFFFFFF010000000000000000D3
:1030040000008001000000000000000000008001BA
:10301400000000000000000000008001000000002B
:10302400000000000000800100000000000000001B
:10303400000080010000000000000000000080FF8C
:10304400FFFFFFFFFFFFFFFFFFFFFF000004024041
:103054004000000006000A000004024004000000D2
:1030640002000900000802400002000009000900F3
:1030740000080240000400000A00090000080240A1
:1030840000010000080009000000024002000000E6
:1030940001000900005C0040000002400001000043
:1030A40008000400000402400001000008000900B8
:1030B40000008000801A060000400000484900001B
:1030C400000000000000000001000300820007006F
:1030D4008400070001000300020003004000030015
:1030E400800007008400070000000008004000087A
:1030F4000080000800C00008000001080000020869
:1031040000000408000006080000080800000A087F
:1031140000000C0800000E08000008001000180051
:1031240020002800300038004000480050005800BB
:10313400000000006410B71DC8206E3BAC30D926D7
:103144009041DC76F4516B6B5861B24D3C71055083
:103154002083B8ED44930FF0E8A3D6D68CB361CBAB
:10316400B0C2649BD4D2D38678E20AA01CF2BDBD5F
:10317400537475636B20627574746F6E2072656727
:10318400697374657220697320696E76616C696411
:103194002C20636C656172696E672E0042757474CD
:1031A4006F6E2069642000697320737475636B21EA
:1031B40000427574746F6E20776173207075736844
:1031C4006564206F6E20626F6F742E204275747474
:1031D4006F6E20636F756E7465723A20004261638E
:1031E4006B0055700053656C65637400446F776EB3
:1031F400002E2E2F7372632F647269766572732F9B
:103204006932632E630049324320646576696365DD
:10321400204944206F7574206F6620626F756E6458
:103224007320256420286D61783A20256429006F75
:103234006E002E2E2F7372632F647269766572731B
:103244002F706D69632F617333373031622E6300E1
:103254004661696C656420746F20737461727420B4
:10326400504D494320313230487A2050574D002088
:103274006973206F757473696465207379737465F9
:103284006D20666C617368006661696C65642074A6
:103294006F20657261736520736563746F722000BB
:1032A4006661696C656420746F2077726974652047
:1032B400616464726573732000496E76616C69643D
:1032C400206669726D7761726520646573637269E3
:1032D4007074696F6E2100436865636B73756D6DFF
:1032E400696E67206669726D7761726520757064B6
:1032F4006174650043616C63756C6174656420631B
:103304006865636B73756D3A2000496E76616C690C
:1033140064206669726D7761726520435243206947
:103324006E2053504920666C617368210065726198
:1033340073655F6F6C645F6669726D776172650057
:1033440077726974655F6E65775F6669726D7761C0
:10335400726500576527726520646561640043687F
:1033640065636B73756D6D696E6720002062797497
:1033740065730D0A00436865636B73756D202D20BA
:1033840077616E746564200020676F7420004F7548
:103394007220696E7465726E616C20666C6173680C
:1033A40020636F6E74656E74732061726520626150
:1033B400642028636865636B73756D206661696C4E
:1033C40065642921205468697320697320726561DA
:1033D4006C6C792062616421004F75722070726593
:1033E40076696F7573206669726D77617265207591
:1033F4007064617465206661696C65642C20616227
:103404006F7274696E67207570646174652E004E06
:103414006577206669726D776172652069732061D2
:103424007661696C61626C6521004C6F6164696EE0
:1034340067207265636F76657279206669726D774D
:10344400617265004661696C656420746F206C6FFD
:103454006164207265636F76657279206669726D46
:10346400776172652C20737472696B65206F6E6569
:103474002E2054727920616761696E2E004661695D
:103484006C656420746F206C6F6164207265636F77
:1034940076657279206669726D776172652C207326
:1034A4007472696B652074776F2E20547279206171
:1034B4006761696E2E004661696C656420746F20D3
:1034C4006C6F6164207265636F76657279206669DA
:1034D400726D776172652C20737472696B652074E8
:1034E400687265652E205341442057415443480077
:1034F40048415244204641554C5400657869742033
:103504007374616E64627900205F5F5F20205F20C6
:10351400205F20205F202020002F205F5F3E3C5F43
:103524003E7C207C7C207C5F5F005C5F5F205C7C59
:10353400207C7C207C7C202F202F003C5F5F5F2F31
:103544007C5F7C7C5F7C7C5F5C5F5C0069326320B9
:10355400696E6974656400706D696320696E69746D
:10356400656400626F6F7420626974004C617374E7
:10357400206669726D7761726520626F6F7420775F
:10358400617320737461626C653B20636C65617266
:1035940020737472696B657300504D494320776FD3
:1035A4006B652066726F6D207374616E646279203E
:1035B40064756520746F2063686172676572206446
:1035C4006973636F6E6E6563740050757474696EAD
:1035D4006720504D4943206261636B20696E746FAC
:1035E400207374616E64627900486F6C6420646F48
:1035F400776E205550202B204241434B202B2053E3
:10360400454C45435420666F7220352073656373BF
:103614002E20746F20666F7263652D626F6F742045
:10362400505246004669726D776172652069732055
:10363400657261736564005761746368646F6720C1
:1036440063617573656420612072657365740053EA
:103654006F667477617265206661696C7572652046
:1036640063617573656420612072657365740046D7
:1036740061696C656420746F207374617274206670
:1036840069726D776172652C20737472696B652041
:1036940074687265652E004661696C656420746F98
:1036A400207374617274206669726D776172652C1F
:1036B40020737472696B652074776F2E004661699C
:1036C4006C656420746F207374617274206669720F
:1036D4006D776172652C20737472696B65206F6EEF
:1036E400652E0053687574646F776E20726571750A
:1036F40065737465642E0052656D6F76652063682A
:10370400617267657220746F2073687574646F7773
:103714006E005368757474696E6720646F776E2EDB
:1037240000426F6F74696E67206669726D776172AB
:1037340065204020002E2E2E0D0A0D0A00466F72C1
:1037440063652D626F6F74696E67207265636F764F
:10375400657279206D6F64652E2E2E00426F6F7432
:1037640020626974733A20004153534552543A20FD
:10377400003A004153534552540041535345525467
:103784004E002A2A2A20575446200053544D3332DF
:103794000053544D333220706572697068657261EC
:1037A4006C206C69627261727920747269707065E0
:1037B4006420616E206173736572740043524F41DB
:1037C4004B204F4F4D0069746F61206275666665CA
:0C37D4007220746F6F20736D616C6C00CC
:1037E000FFFFFFFF008400000202000000C0040190
:1037F00000000000000000021000000007000000B0
:103800000000010203040102030406070809000086
:04000005080001846A
:00000001FF
